:020000040000FA
:0408000030EF05F0E0
:1008100003B23DEF04F0F2B458EF04F09EB060EF85
:1008200004F09EB268EF04F0F2A81AEF04F0F2B2FE
:100830001CEF04F00EEF05F0CD90F29207BC078E8E
:10084000078C9EA029EF04F00101463F29EF04F038
:10085000472B07AE34EF04F0CECF51F1CFCF52F19A
:1008600046C153F147C154F1CF6ACE6A0101466BCC
:10087000476B9E90CD800EEF05F00392030103EECF
:1008800000F080517F0BE92604C0EFFF802B8151DF
:10089000805D700BD8A48B8200008051815D700B4D
:1008A000D8A48B9281518019D8B407900EEF05F02F
:1008B000F2940101383F0EEF05F0392B0EEF05F0F1
:1008C0009E900101463F0EEF05F0472B0EEF05F01D
:1008D0009E92C3CF48F1C4CF49F1C28207B492EFD0
:1008E00004F03AC13EF13BC13FF13CC140F13DC192
:1008F00041F151C155F152C156F153C157F154C1A3
:1009000058F1010148514E2749514F23E86A5023BD
:100910000D2E92EF04F04FC14AF150C14BF14E6BD6
:100920004F6B506B0201002F0EEF05F03C0E006F75
:1009300001015D67A3EF04F05E67A3EF04F05F675A
:10094000A3EF04F06067A7EF04F0D7EF04F061C1F4
:1009500000F162C101F163C102F164C103F101015F
:10096000010E046F000E056F000E066F000E076F7C
:10097000B8EC11F000C161F101C162F102C163F193
:1009800003C164F10067CCEF04F00167CCEF04F021
:100990000267CCEF04F00367D7EF04F05DC161F1AB
:1009A0005EC162F15FC163F160C164F10E80D57E0A
:1009B000D5BE32D0D6CF3AF1D7CF3BF138C13CF1DA
:1009C000E86AE8CF3DF1010147A7F2EF04F0079C88
:1009D000079E0101000E516F600E526F3D0E536F66
:1009E000080E546F01013ABF02EF05F03B6702EFBA
:1009F00005F03C6702EF05F03D6702EF05F0F28875
:100A000007EF05F0F298516B526B536B546BD76A3A
:100A1000D66A0101386B396B0EEF05F002C0E0FFBA
:100A2000005001C0D8FF1000A6B214EF05F00CC0B2
:100A3000A9FF0BC0A8FFA69EA69CA684F29E550EF9
:100A4000A76EAA0EA76EA682F28EA694A6B226EF75
:100A500005F01200A96EA69EA69CA680A8501200C2
:100A6000076A0E6A0F010E0EC16E860EC06E030E6F
:100A7000C26E0F01896A110E926E080E8A6EF10E17
:100A8000936E8B6A800E946EF18E0D6A4E6B4F6B77
:100A9000506B4A6B4B6B0F01280ED56EF28AB00E6D
:100AA000CD6E9D800101516B526B536B546B556B36
:100AB000566B576B586B596B5A6B5B6B5C6B079C37
:100AC000079E760ECA6E9D8202013C0E006FCC6AB4
:100AD000160E2AEC05F0E8CF00F1170E2AEC05F00F
:100AE000E8CF01F1180E2AEC05F0E8CF02F1190E5B
:100AF0002AEC05F0E8CF03F1010103AF9AEF05F00E
:100B0000AFEC12F0160E0C6E00C10BF014EC05F0F9
:100B1000170E0C6E01C10BF014EC05F0180E0C6EE4
:100B200002C10BF014EC05F0190E0C6E03C10BF0B2
:100B300014EC05F000C15DF101C15EF102C15FF18D
:100B400003C160F100C161F101C162F102C163F151
:100B500003C164F11A0E2AEC05F0E8CF00F11B0E78
:100B60002AEC05F0E8CF01F11C0E2AEC05F0E8CFE5
:100B700002F11D0E2AEC05F0E8CF03F1010103AFED
:100B8000F0EF05F0AFEC12F01A0E0C6E00C10BF096
:100B900014EC05F01B0E0C6E01C10BF014EC05F00B
:100BA0001C0E0C6E02C10BF014EC05F01D0E0C6E49
:100BB00003C10BF014EC05F01A0E2AEC05F0E8CF97
:100BC00000F11B0E2AEC05F0E8CF01F11C0E2AEC17
:100BD00005F0E8CF02F11D0E2AEC05F0E8CF03F195
:100BE00000C165F101C166F102C167F103C168F19D
:100BF000240EAC6E0401806B816B0F01900EAB6E06
:100C00000F019D8A0301806B816BA26B8B92079011
:100C10000001F28EF28C07B0C3EF0FF00EB08AEF36
:100C20000AF00301805181197F0BD8B4C3EF0FF094
:100C300013EE00F081517F0BE126812BE7CFE8FF17
:100C4000E00BD8B4C3EF0FF023EE82F0A2511F0BDC
:100C5000D926E7CFDFFFA22BDF50780AD8A4C3EF55
:100C60000FF0078061C100F162C101F163C102F1BF
:100C700064C103F10101040E046F000E056F000E44
:100C8000066F000E076FB8EC11F000AF51EF06F0E1
:100C90000101030E616F000E626F000E636F000EA4
:100CA000646F03018251720AD8B48AEF0AF082514C
:100CB000630AD8B483EF0CF08251690AD8B45FEFAD
:100CC00008F082517A0AD8B472EF09F08251490AC9
:100CD000D8B476EF07F08251500AD8B494EF06F0FA
:100CE0008251700AD8B4D7EF06F08251540AD8B4B2
:100CF00002EF07F08251740AD8B448EF07F0B8EF5A
:100D00000CF0040114EE00F080517F0BE12682C448
:100D1000E7FF802B12000D0E826F81EC06F00A0EA9
:100D2000826F81EC06F0120083C31EF184C31FF1B1
:100D300085C320F186C321F187C322F188C323F143
:100D400089C324F18AC325F18BC326F18CC327F113
:100D50000101FCEC12F074EC12F0160E0C6E00C1E6
:100D60000BF014EC05F0170E0C6E01C10BF014EC37
:100D700005F0180E0C6E02C10BF014EC05F0190E04
:100D80000C6E03C10BF014EC05F000C15DF101C164
:100D90005EF102C15FF103C160F100C161F101C107
:100DA00062F102C163F103C164F176EF07F083C31E
:100DB0001EF184C31FF185C320F186C321F187C3CF
:100DC00022F188C323F189C324F18AC325F18BC39F
:100DD00026F18CC327F10101FCEC12F074EC12F047
:100DE00000C15DF101C15EF102C15FF103C160F1BB
:100DF00000C161F101C162F102C163F103C164F19B
:100E000076EF07F083C31EF184C31FF185C320F181
:100E100086C321F187C322F188C323F189C324F15A
:100E20008AC325F18CC326F18DC327F10101FCECA7
:100E300012F074EC12F00101000E046F000E056F49
:100E4000010E066F000E076FC7EC11F01A0E0C6E44
:100E500000C10BF014EC05F01B0E0C6E01C10BF081
:100E600014EC05F01C0E0C6E02C10BF014EC05F036
:100E70001D0E0C6E03C10BF014EC05F000C165F102
:100E800001C166F102C167F103C168F176EF07F0B5
:100E900083C31EF184C31FF185C320F186C321F1F2
:100EA00087C322F188C323F189C324F18AC325F1C2
:100EB0008CC326F18DC327F10101FCEC12F074EC18
:100EC00012F00101000E046F000E056F010E066F97
:100ED000000E076FC7EC11F000C165F101C166F1AA
:100EE00002C167F103C168F176EF07F0160E2AEC34
:100EF00005F0E8CF00F1170E2AEC05F0E8CF01F17C
:100F0000180E2AEC05F0E8CF02F1190E2AEC05F0D4
:100F1000E8CF03F152EC12F01EC182F40401300E4E
:100F2000822781EC06F01FC182F40401300E822773
:100F300081EC06F020C182F40401300E822781EC9E
:100F400006F021C182F40401300E822781EC06F004
:100F500022C182F40401300E822781EC06F023C105
:100F600082F40401300E822781EC06F024C182F461
:100F70000401300E822781EC06F025C182F40401C1
:100F8000300E822781EC06F026C182F40401300E77
:100F9000822781EC06F027C182F40401300E8227FB
:100FA00081EC06F00401730E826F81EC06F00401FF
:100FB0002C0E826F81EC06F05DC100F15EC101F183
:100FC0005FC102F160C103F152EC12F01EC182F464
:100FD0000401300E822781EC06F01FC182F4040167
:100FE000300E822781EC06F020C182F40401300E1D
:100FF000822781EC06F021C182F40401300E8227A1
:1010000081EC06F022C182F40401300E822781ECCB
:1010100006F023C182F40401300E822781EC06F031
:1010200024C182F40401300E822781EC06F025C130
:1010300082F40401300E822781EC06F026C182F48E
:101040000401300E822781EC06F027C182F40401EE
:10105000300E822781EC06F00401730E826F81EC62
:1010600006F004012C0E826F81EC06F01A0E2AECB9
:1010700005F0E8CF00F11B0E2AEC05F0E8CF01F1F6
:101080001C0E2AEC05F0E8CF02F11D0E2AEC05F04B
:10109000E8CF03F1D2EC0CF004012C0E826F81EC4E
:1010A00006F065C100F166C101F167C102F168C1D6
:1010B00003F1D2EC0CF08BEC06F0B8EF0CF004016D
:1010C000690E826F81EC06F004012C0E826F81ECB8
:1010D00006F00101040E006F000E016F000E026F9A
:1010E000000E036F52EC12F020C182F40401300EA6
:1010F000822781EC06F021C182F40401300E8227A0
:1011000081EC06F022C182F40401300E822781ECCA
:1011100006F023C182F40401300E822781EC06F030
:1011200024C182F40401300E822781EC06F025C12F
:1011300082F40401300E822781EC06F026C182F48D
:101140000401300E822781EC06F027C182F40401ED
:10115000300E822781EC06F004012C0E826F81ECA8
:1011600006F00101030E006F000E016F000E026F0A
:10117000000E036F52EC12F020C182F40401300E15
:10118000822781EC06F021C182F40401300E82270F
:1011900081EC06F022C182F40401300E822781EC3A
:1011A00006F023C182F40401300E822781EC06F0A0
:1011B00024C182F40401300E822781EC06F025C19F
:1011C00082F40401300E822781EC06F026C182F4FD
:1011D0000401300E822781EC06F027C182F404015D
:1011E000300E822781EC06F004012C0E826F81EC18
:1011F00006F001010E0E006F000E016F000E026F6F
:10120000000E036F52EC12F020C182F40401300E84
:10121000822781EC06F021C182F40401300E82277E
:1012200081EC06F022C182F40401300E822781ECA9
:1012300006F023C182F40401300E822781EC06F00F
:1012400024C182F40401300E822781EC06F025C10E
:1012500082F40401300E822781EC06F026C182F46C
:101260000401300E822781EC06F027C182F40401CC
:10127000300E822781EC06F004012C0E826F81EC87
:1012800006F0200EF86EF76AF66A04010900F5CF41
:1012900082F481EC06F00900F5CF82F481EC06F0CF
:1012A0000900F5CF82F481EC06F00900F5CF82F455
:1012B00081EC06F00900F5CF82F481EC06F009001C
:1012C000F5CF82F481EC06F00900F5CF82F481ECD1
:1012D00006F00900F5CF82F481EC06F08BEC06F005
:1012E000B8EF0CF08351630AD8A4B8EF0CF0845126
:1012F000610AD8A4B8EF0CF085516C0AD8A4B8EFF5
:101300000CF08651410A42E08651440A1BE08651A6
:10131000420AD8B4D9EF09F08651350AD8B441EF62
:101320000EF08651360AD8B495EF0EF08651370A82
:10133000D8B4FDEF0EF08651380AD8B45BEF0FF049
:10134000B8EF0CF00798079A04017A0E826F81ECCF
:1013500006F00401780E826F81EC06F00401640E41
:10136000826F81EC06F081A8BDEF09F00401550EF3
:10137000826F81EC06F0C2EF09F004014C0E826F1F
:1013800081EC06F08BEC06F0B8EF0CF00788079ABA
:1013900004017A0E826F81EC06F00401410E826F27
:1013A00081EC06F00401610E826F81EC06F0B3EF70
:1013B00009F00798078A04017A0E826F81EC06F023
:1013C0000401420E826F81EC06F00401610E826F0F
:1013D00081EC06F0B3EF09F00101620E046F010E1B
:1013E000056F000E066F000E076F59C100F15AC15C
:1013F00001F15BC102F15CC103F1B8EC11F003BF74
:1014000049EF0AF00E0E2AEC05F0E8CF0CF10F0EB2
:101410002AEC05F0E8CF0DF1100E2AEC05F0E8CF2C
:101420000EF1110E2AEC05F0E8CF0FF101EC11F0EE
:1014300059C104F15AC105F15BC106F15CC107F164
:10144000B8EC11F00782C5EC10F001EC11F0079236
:10145000C5EC10F059C100F15AC101F15BC102F1B4
:101460005CC103F10792C5EC10F0CC0E046FE00EE6
:10147000056F870E066F050E076FB8EC11F000C1FF
:101480000CF101C10DF102C10EF103C10FF181EFA9
:101490000AF00101800E006F1A0E016F060E026F36
:1014A000000E036F42C104F143C105F144C106F1CE
:1014B00045C107F1B8EC11F003AF62EF0AF0AFECF1
:1014C00012F012000E0E2AEC05F0E8CF0CF10F0E10
:1014D0002AEC05F0E8CF0DF1100E2AEC05F0E8CF6C
:1014E0000EF1110E2AEC05F0E8CF0FF142C100F128
:1014F00043C101F144C102F145C103F10782C5ECCA
:1015000010F00CC100F10DC101F10EC102F10FC1CB
:1015100003F11200078455C159F156C15AF157C160
:101520005BF158C15CF13EC142F13FC143F140C1A2
:1015300044F141C145F14AC14CF14BC14DF1079411
:101540000EA0C1EF0AF001016567AEEF0AF0666711
:10155000AEEF0AF06767AEEF0AF06867B2EF0AF025
:10156000C1EF0AF0ECEC09F065C104F166C105F1C8
:1015700067C106F168C107F1B8EC11F003BF80EF55
:101580000CF0ECEC09F00101000E046F000E056F89
:10159000010E066F000E076FE6EC11F00401720EEB
:1015A000826F81EC06F004012C0E826F81EC06F054
:1015B00052EC12F01D67E2EF0AF00401200E826F78
:1015C000E5EF0AF004012D0E826F81EC06F024C1D4
:1015D00082F40401300E822781EC06F025C182F4EA
:1015E0000401300E822781EC06F004012E0E826F7A
:1015F00081EC06F026C182F40401300E822781ECD2
:1016000006F027C182F40401300E822781EC06F037
:1016100004016D0E826F81EC06F004012C0E826FC6
:1016200081EC06F042C100F143C101F144C102F175
:1016300045C103F1010152EC12F01EC182F4040114
:10164000300E822781EC06F01FC182F40401300EB7
:10165000822781EC06F020C182F40401300E82273B
:1016600081EC06F021C182F40401300E822781EC66
:1016700006F022C182F40401300E822781EC06F0CC
:1016800023C182F40401300E822781EC06F024C1CC
:1016900082F40401300E822781EC06F025C182F429
:1016A0000401300E822781EC06F026C182F4040189
:1016B000300E822781EC06F027C182F40401300E3F
:1016C000822781EC06F00401480E826F81EC06F05F
:1016D00004017A0E826F81EC06F004012C0E826FF9
:1016E00081EC06F059C100F15AC101F15BC102F170
:1016F0005CC103F1010152EC12F01EC182F404013D
:10170000300E822781EC06F01FC182F40401300EF6
:10171000822781EC06F020C182F40401300E82277A
:1017200081EC06F021C182F40401300E822781ECA5
:1017300006F022C182F40401300E822781EC06F00B
:1017400023C182F40401300E822781EC06F024C10B
:1017500082F40401300E822781EC06F025C182F468
:101760000401300E822781EC06F026C182F40401C8
:10177000300E822781EC06F027C182F40401300E7E
:10178000822781EC06F00401630E826F81EC06F083
:1017900004012C0E826F81EC06F059C100F15AC190
:1017A00001F15BC102F15CC103F101010A0E046F9A
:1017B000000E056F000E066F000E076FC7EC11F0EC
:1017C000000E046F120E056F000E066F000E076FFD
:1017D000E6EC11F052EC12F01EC182F40401300E5E
:1017E000822781EC06F01FC182F40401300E8227AB
:1017F00081EC06F020C182F40401300E822781ECD6
:1018000006F021C182F40401300E822781EC06F03B
:1018100022C182F40401300E822781EC06F023C13C
:1018200082F40401300E822781EC06F024C182F498
:101830000401300E822781EC06F004012E0E826F27
:1018400081EC06F025C182F40401300E822781EC80
:1018500006F026C182F40401300E822781EC06F0E6
:1018600027C182F40401300E822781EC06F00401C6
:10187000730E826F81EC06F004012C0E826F81ECF6
:1018800006F0AFEC12F04CC100F14DC101F1E1ECFA
:101890000DF00EA07EEF0CF004012C0E826F81EC97
:1018A00006F0200EF86EF76AF66A04010900F5CF1B
:1018B00082F481EC06F00900F5CF82F481EC06F0A9
:1018C0000900F5CF82F481EC06F00900F5CF82F42F
:1018D00081EC06F00900F5CF82F481EC06F00900F6
:1018E000F5CF82F481EC06F00900F5CF82F481ECAB
:1018F00006F00900F5CF82F481EC06F08BEC06F0DF
:101900000E90B8EF0CF00401630E826F81EC06F0CC
:1019100004012C0E826F81EC06F0BDEC0CF004018A
:101920002C0E826F81EC06F030EC0DF004012C0ED1
:10193000826F81EC06F0ACEC0DF004012C0E826F8E
:1019400081EC06F00101F80E006FCD0E016F660EFE
:10195000026F030E036FD2EC0CF004012C0E826FA9
:1019600081EC06F0C2EC0DF08BEC06F0B8EF0CF059
:101970000301A26B0790C3EF0FF0D8900E0E2AEC74
:1019800005F0E8CF00F10F0E2AEC05F0E8CF01F1E9
:10199000100E2AEC05F0E8CF02F1110E2AEC05F04A
:1019A000E8CF03F10101000E046F000E056F010E78
:1019B000066F000E076FE6EC11F052EC12F01EC13C
:1019C00082F40401300E822781EC06F01FC182F4FC
:1019D0000401300E822781EC06F020C182F404015C
:1019E000300E822781EC06F021C182F40401300E12
:1019F000822781EC06F022C182F40401300E822796
:101A000081EC06F023C182F40401300E822781ECC0
:101A100006F024C182F40401300E822781EC06F026
:101A200025C182F40401300E822781EC06F0040106
:101A30002E0E826F81EC06F026C182F40401300E76
:101A4000822781EC06F027C182F40401300E822740
:101A500081EC06F004016D0E826F81EC06F012003D
:101A6000120E2AEC05F0E8CF00F1130E2AEC05F077
:101A7000E8CF01F1140E2AEC05F0E8CF02F1150EC3
:101A80002AEC05F0E8CF03F101010A0E046F000E05
:101A9000056F000E066F000E076FC7EC11F0000E09
:101AA000046F120E056F000E066F000E076FE6EC56
:101AB00011F052EC12F01EC182F40401300E8227A4
:101AC00081EC06F01FC182F40401300E822781EC04
:101AD00006F020C182F40401300E822781EC06F06A
:101AE00021C182F40401300E822781EC06F022C16C
:101AF00082F40401300E822781EC06F023C182F4C7
:101B00000401300E822781EC06F024C182F4040126
:101B1000300E822781EC06F004012E0E826F81ECDC
:101B200006F025C182F40401300E822781EC06F014
:101B300026C182F40401300E822781EC06F027C111
:101B400082F40401300E822781EC06F00401730E4A
:101B5000826F81EC06F012000A0E2AEC05F0E8CF45
:101B600000F10B0E2AEC05F0E8CF01F10C0E2AEC87
:101B700005F0E8CF02F10D0E2AEC05F0E8CF03F1F5
:101B8000E1EF0DF0060E2AEC05F0E8CF00F1070EAC
:101B90002AEC05F0E8CF01F1080E2AEC05F0E8CFB9
:101BA00002F1090E2AEC05F0E8CF03F1E1EF0DF0A8
:101BB0000101AFEC12F007844AC100F14BC101F101
:101BC00007940101E80E046F800E056F000E066F8A
:101BD000000E076FC7EC11F0000E046F040E056FC6
:101BE000000E066F000E076FE6EC11F0880E046F12
:101BF000130E056F000E066F000E076FB8EC11F0A4
:101C00000A0E046F000E056F000E066F000E076FC0
:101C1000E6EC11F052EC12F001011D6715EF0EF029
:101C20000401200E826F18EF0EF004012D0E826F5A
:101C300081EC06F024C182F40401300E822781EC8D
:101C400006F025C182F40401300E822781EC06F0F3
:101C500026C182F40401300E822781EC06F00401D3
:101C60002E0E826F81EC06F027C182F40401300E43
:101C7000822781EC06F00401430E826F81EC06F0AE
:101C8000120087C31EF188C31FF189C320F18AC3E4
:101C900021F18BC322F18CC323F18DC324F18EC3B8
:101CA00025F190C326F191C327F10101FCEC12F05C
:101CB00074EC12F00101000E046F000E056F010EAE
:101CC000066F000E076FC7EC11F00E0E0C6E00C110
:101CD0000BF014EC05F00F0E0C6E01C10BF014ECC0
:101CE00005F0100E0C6E02C10BF014EC05F0110E95
:101CF0000C6E03C10BF014EC05F004017A0E826F38
:101D000081EC06F004012C0E826F81EC06F00401D8
:101D1000350E826F81EC06F004012C0E826F81EC8F
:101D200006F0BDEC0CF0C2EF09F087C31EF188C3CA
:101D30001FF189C320F18AC321F18BC322F18CC327
:101D400023F18DC324F18EC325F190C326F191C3F5
:101D500027F10101FCEC12F074EC12F0880E046F14
:101D6000130E056F000E066F000E076FBCEC11F02E
:101D7000000E046F040E056F000E066F000E076F55
:101D8000C7EC11F00101E80E046F800E056F000E24
:101D9000066F000E076FE6EC11F00A0E0C6E00C124
:101DA0000BF014EC05F00B0E0C6E01C10BF014ECF3
:101DB00005F00C0E0C6E02C10BF014EC05F00D0ECC
:101DC0000C6E03C10BF014EC05F004017A0E826F67
:101DD00081EC06F004012C0E826F81EC06F0040108
:101DE000360E826F81EC06F004012C0E826F81ECBE
:101DF00006F0ACEC0DF0C2EF09F087C31EF188C30A
:101E00001FF189C320F18AC321F18BC322F18CC356
:101E100023F18DC324F18FC325F190C326F191C323
:101E200027F10101FCEC12F074EC12F0000E046FCB
:101E3000120E056F000E066F000E076FC7EC11F053
:101E400001010A0E046F000E056F000E066F000EF2
:101E5000076FE6EC11F0120E0C6E00C10BF014ECE3
:101E600005F0130E0C6E01C10BF014EC05F0140E0E
:101E70000C6E02C10BF014EC05F0150E0C6E03C1D4
:101E80000BF014EC05F004017A0E826F81EC06F081
:101E900004012C0E826F81EC06F00401370E826F74
:101EA00081EC06F004012C0E826F81EC06F030EC20
:101EB0000DF0C2EF09F087C31EF188C31FF189C37B
:101EC00020F18AC321F18BC322F18CC323F18DC38E
:101ED00024F18EC325F190C326F191C327F10101AE
:101EE000FCEC12F074EC12F0880E046F130E056F08
:101EF000000E066F000E076FBCEC11F0000E046FB1
:101F0000040E056F000E066F000E076FC7EC11F090
:101F10000101E80E046F800E056F000E066F000EC3
:101F2000076FE6EC11F0060E0C6E00C10BF014EC1E
:101F300005F0070E0C6E01C10BF014EC05F0080E55
:101F40000C6E02C10BF014EC05F0090E0C6E03C10F
:101F50000BF014EC05F004017A0E826F81EC06F0B0
:101F600004012C0E826F81EC06F00401380E826FA2
:101F700081EC06F004012C0E826F81EC06F0C2ECBD
:101F80000DF0C2EF09F081A881EF10F007A83AEF39
:101F900010F00101800E006F1A0E016F060E026F25
:101FA000000E036F3EC104F13FC105F140C106F1CF
:101FB00041C107F1B8EC11F003BF81EF10F0BFECA5
:101FC00010F03EC100F13FC101F140C102F141C139
:101FD00003F10782C5EC10F00CC104F10DC105F14D
:101FE0000EC106F10FC107F1F80E006FCD0E016FA3
:101FF000660E026F030E036FB8EC11F00E0E0C6E3E
:1020000000C10BF014EC05F00F0E0C6E01C10BF0CB
:1020100014EC05F0100E0C6E02C10BF014EC05F080
:10202000110E0C6E03C10BF014EC05F007840101D6
:10203000AFEC12F04AC100F14BC101F107940A0E56
:102040000C6E00C10BF014EC05F00B0E0C6E01C110
:102050000BF014EC05F00C0E0C6E02C10BF014EC3E
:1020600005F00D0E0C6E03C10BF014EC05F0079893
:1020700081EF10F007AA81EF10F007840101AFECA7
:1020800012F04AC100F14BC101F10794060E0C6E2B
:1020900000C10BF014EC05F0070E0C6E01C10BF043
:1020A00014EC05F0080E0C6E02C10BF014EC05F0F8
:1020B000090E0C6E03C10BF014EC05F0078455C13A
:1020C00000F156C101F157C102F158C103F1079463
:1020D000120E0C6E00C10BF014EC05F0130E0C6E1A
:1020E00001C10BF014EC05F0140E0C6E02C10BF0E4
:1020F00014EC05F0150E0C6E03C10BF014EC05F09A
:10210000079A0401805181197F0B0BE09EA809D02A
:1021100014EE00F081517F0BE126E750812B0F0177
:10212000AD6E0BEF06F00CC100F10DC101F10EC157
:1021300002F10FC103F1000E046F000E056F010ED6
:10214000066F000E076FE6EC11F01DA1BEEF10F058
:102150001451D8B4BEEF10F00CC100F10DC101F163
:102160000EC102F10FC103F1000E046F000E056FE6
:102170000A0E066F000E076FE6EC11F01200010167
:102180000C6B0D6B0E6B0F6B12000101005305E120
:10219000015303E1025301E1002B88EC11F0AFEC95
:1021A00012F02C51006F2D51016F420E046F4B0E37
:1021B000056F000E066F000E076FC7EC11F000C12F
:1021C00004F101C105F102C106F103C107F10CC11F
:1021D00000F10DC101F10EC102F10FC103F107B20F
:1021E000F6EF10F0BCEC11F0F8EF10F0B8EC11F0D5
:1021F00000C10CF101C10DF102C10EF103C10FF1DB
:102200001200AFEC12F04CC100F14DC101F1060E0D
:102210002AEC05F0E8CF04F1070E2AEC05F0E8CF30
:1022200005F1080E2AEC05F0E8CF06F1090E2AECBC
:1022300005F0E8CF07F1B8EC11F000C118F101C1C9
:1022400019F102C11AF103C11BF1290E046F000E2E
:10225000056F000E066F000E076FC7EC11F0EE0E53
:10226000046F430E056F000E066F000E076FBCEC87
:1022700011F018C104F119C105F11AC106F11BC111
:1022800007F1C7EC11F000C110F101C111F102C159
:1022900012F103C113F1120E2AEC05F0E8CF04F19C
:1022A000130E2AEC05F0E8CF05F1140E2AEC05F028
:1022B000E8CF06F1150E2AEC05F0E8CF07F10D0E78
:1022C000006F000E016F000E026F000E036FC7EC6F
:1022D00011F0180E046F000E056F000E066F000E51
:1022E000076FE6EC11F010C104F111C105F112C144
:1022F00006F113C107F1BCEC11F06A0E046F2A0E4F
:10230000056F000E066F000E076FB8EC11F012009B
:10231000BF0EFA6E200E2D6F2C6BD8900037013750
:1023200002370337D8B099EF11F02D2F8EEF11F04F
:102330002C072D070353D8B412000331070B800973
:10234000326F03390F0B010F2C6F80EC5FF0336F8E
:102350002C0580EC5FF0335D335F2C6B3233D8B0EB
:102360002C272C3332A9AEEF11F033512C27120059
:10237000D4EC12F0D8B0120003510719286F97EC73
:1023800012F0D8900751031928AF800F1200286B64
:10239000BBEC12F0D8A0D1EC12F0D8B01200A6EC31
:1023A00012F0AFEC12F01F0E296FE7EC12F00B35B4
:1023B000D8B097EC12F0D8A00335D8B01200292F6E
:1023C000D5EF11F028B1BEEC12F01200286B0451C9
:1023D0000511061107110008D8A0BBEC12F0D8A017
:1023E000D1EC12F0D8B01200086B096B0A6B0B6BC2
:1023F000E7EC12F01F0E296FE7EC12F007510B5DAE
:10240000D8A40FEF12F006510A5DD8A40FEF12F016
:102410000551095DD8A40FEF12F00451085DD8A052
:1024200022EF12F00451085F0551D8A0053D095F65
:102430000651D8A0063D0A5F0751D8A0073D0B5FA3
:10244000D8900081292FFCEF11F028B1BEEC12F0DA
:10245000286BBBEC12F0D890EBEC12F007510B5D3F
:10246000D8A43FEF12F006510A5DD8A43FEF12F056
:102470000551095DD8A43FEF12F00451085DD8A0C2
:102480004EEF12F0003F4EEF12F0013F4EEF12F010
:10249000023F4EEF12F0032BD8B4120028B1BEEC6D
:1024A00012F012000101286BBBEC12F0D8B0120040
:1024B000F0EC12F0200E296F003701370237033796
:1024C00011EE27F00A0E2A6FE7360A0EE75CD8B045
:1024D000E76EE5522A2F64EF12F0292F5CEF12F01D
:1024E00028B11D81D890120001010A0E286F200E1C
:1024F000296F11EE1DF028512A6F0A0ED890E6526E
:10250000D8B0E726E7322A2F7FEF12F003330233E9
:1025100001330033292F79EF12F0E750FF0FD8A0D5
:102520000335D8B012001DB1BEEC12F012000451F8
:1025300000270551D8B0053D01270651D8B0063D0A
:1025400002270751D8B0073D032712000051086F3A
:102550000151096F02510A6F03510B6F1200010103
:10256000006B016B026B036B12000101046B056BC6
:10257000066B076B12000335D8A012000351800BC5
:10258000001F011F021F031F003FCEEF12F0013F8B
:10259000CEEF12F0023FCEEF12F0032B282B0325D3
:1025A00012000735D8A012000751800B041F051F29
:1025B000061F071F043FE4EF12F0053FE4EF12F09F
:1025C000063FE4EF12F0072B282B072512000037F7
:1025D000013702370337083709370A370B3712003C
:1025E0001D6B1E6B1F6B206B216B226B236B246B8F
:1025F000256B266B276B12001E510F0B1E6F1F5190
:102600000F0B1F6F20510F0B206F21510F0B216FEC
:1026100022510F0B226F23510F0B236F24510F0BED
:10262000246F25510F0B256F26510F0B266F275155
:062630000F0B276F1200E2
:10BF0000E844F926000C160C2B0C3F0C520C640C68
:10BF1000760C860C960CA50CB30CC10CCF0CDC0C6B
:06BF2000E80CF40C000C1B
:00000001FF
